:100000000C94C5020C94FD020C94FD020C94FD02AC
:100010000C94FD020C94FD020C94FD020C94FD0264
:100020000C94FD020C94FD020C94F0280C94C2294F
:100030000C94CF230C94FD020C94FD020C94FD0251
:100040000C94FD020C94FD020C94FD020C94FD0234
:100050000C94681F0C9457240C94FD020C94FD0220
:100060000C94FD020C94FD020C94FD020C94FD0214
:100070000C94FD020C94FD020C94FD020C94FD0204
:100080000C94FD020C94FD020C94FD020C94FD02F4
:100090000C94FD020C94FD020C94FD020C94FD02E4
:1000A0000C94FD020C94FD020C94FD02C405C405E1
:1000B000F005F005580676068E078E0781061A07AA
:1000C0002B072B07771E791E7E1E811E841E871E1E
:1000D0008A1E2F2A562A4E2B562A4E2BA22AC52A72
:1000E0004E2B1C2B2B2B2900550054002A005F009F
:1000F0006000610056005C005D005E005700590022
:100100005A005B005800620063000151C35C530059
:100110000100010001000100010001000100AC002C
:10012000AE00AB000100AA00A800A9000100005C1D
:10013000025101000100C35CC65CC85CCA5CC45CBF
:10014000C75CC95CCB5CC05CBC5CBF5CC15C0100D3
:10015000BD5CBE5CC25C0100010001000100010049
:100160000100010001000100010001000100010087
:100170000100010001000100010001000100010077
:1001800001000100010000047F3F1F64321464324B
:1001900014783C1E1E140A052223252628292A2C01
:1001A0002D2F3032333536383A3B3D3E40424345C1
:1001B00047494A4C4E5051535557595A5C5E6062FC
:1001C000646668696B6D6F71737577797B7D7F810C
:1001D000838587898A8C8E90929496989A9C9E9F0C
:1001E000A1A3A5A7A8AAACAEAFB1B3B4B6B8B9BB2A
:1001F000BCBEBFC1C2C3C5C6C7C9CACBCCCDCED099
:10020000D1D2D2D3D4D5D6D7D7D8D9D9DADADBDB85
:10021000DBDCDCDCDCDCDDDDDDDDDCDCDCDCDCDB1C
:10022000DBDBDADAD9D9D8D7D7D6D5D4D3D2D2D165
:10023000D0CECDCCCBCAC9C7C6C5C3C2C1BFBEBC58
:10024000BBB9B8B6B4B3B1AFAEACAAA8A7A5A3A1C9
:100250009F9E9C9A98969492908E8C8A898785838B
:10026000817F7D7B79777573716F6D6B696866646B
:1002700062605E5C5A5957555351504E4C4A49473B
:10028000454342403E3D3B3A3836353332302F2DE0
:100290002C2A292826252322FFAA7F55400000006A
:1002A0000000000000000000010102030405060830
:1002B0000A0C0F1114181C2024292E33393F464CE8
:1002C000535B626A7179818A929AA2AAB2B9C1C853
:1002D000CFD5DCE1E7EBF0F4F7FAFCFDFEFFFEFD25
:1002E000FCFAF7F4F0EBE7E1DCD5CFC8C1B9B2AA6C
:1002F000A29A928A8179716A625B534C463F393384
:100300002E2924201C1814110F0C0A0806050403BA
:1003100002010100000000000000000000000101D7
:1003200001010101010101020202020202020202B4
:100330000303030303030303040404040404040584
:100340000505050506060606060707070707080848
:100350000808090909090A0A0A0B0B0B0C0C0C0DF9
:100360000D0D0E0E0E0F0F0F101011111112121392
:10037000131414151516161717181819191A1A1B0D
:100380001B1C1D1D1E1E1F2020212222232424256C
:100390002626272829292A2B2C2D2D2E2F303132A5
:1003A00032333435363738393A3B3C3D3E3F4041B5
:1003B00042434445464748494A4C4D4E4F5051539D
:1003C00054555658595A5B5D5E5F61626465666854
:1003D000696B6C6D6F7072737577787A7B7D7E80D8
:1003E00082838587888A8C8E8F91939596989A9C24
:1003F0009EA0A2A3A5A7A9ABADAFB1B3B5B7BABC38
:10040000BEC0C2C4C6C9CBCDCFD1D4D6D8DBDDDF08
:10041000E2E4E7E9EBEEF0F3F5F8FAFDFF08035349
:10042000003200300000001A0370006F006C007989
:10043000006300610072006200640069006500747E
:100440000000000403090409023B00020100A0FAB5
:10045000090400000103010100092111010001222A
:1004600040000705810308000109040100010300A1
:10047000000009211101000122B6000705820320B6
:10048000000112010002000000084050207301002A
:100490000102000105010902A10185020901A10073
:1004A0000509190129081500250195087501810222
:1004B0000501093009311581257F950275088106EE
:1004C00009381581257F950175088106050C0A38C4
:1004D000021581257F950175088106C0C0050109B7
:1004E00080A101850319012AB700150126B70095DF
:1004F0000175108100C0050C0901A10185041901D5
:100500002AA002150126A002950175108100C005E0
:10051000010906A1018506050719E029E71500254F
:10052000019508750181020507190029EF150025BD
:100530000195F075018102050819012905950575D8
:10054000019102950175039101C005010906A10100
:10055000050719E029E715002501950875018102B5
:100560009501750881010507190029FF150026FF6F
:10057000009506750881000508190129059505757E
:10058000019102950175039101C011241FBECFEFA7
:10059000DAE0DEBFCDBF04B603FE18C08091E402EE
:1005A0009091E502A091E602B091E7028730904B6E
:1005B000A740B04B59F41092E4021092E502109259
:1005C000E6021092E702E0E0F8E3099511E0A0E00E
:1005D000B1E0EEEEF8E502C005900D92AE3BB1073A
:1005E000D9F722E0AEEBB1E001C01D92A43EB20704
:1005F000E1F70E948A130C94752C0C94000081E0A2
:10060000089581E008950C94010308950C94050366
:100610001F93CF93DF9300D000D01F92CDB7DEB7EA
:1006200049835A836B833091C10189819A81311149
:1006300014C0662359F0222349F00E94C909182FDB
:10064000682F89819A810E94740903C00E949E09C3
:10065000182F69817A81812F04C00E94C90969819C
:100660007A810F900F900F900F900F90DF91CF91A4
:100670001F910C94FF10FC01262F40815181628153
:10068000738184810C94080381E00895CF93DF93F4
:10069000EC0160E00E943B03BE01DF91CF910C941E
:1006A00006030C9443120C943F1208950E941E08F6
:1006B0000E9455032FEF84E39CE02150804090403E
:1006C000E1F700C000000C947D240F931F93CF939B
:1006D000DF938C0161E00E943B03EC01B8010E94B2
:1006E0000303882309F44BC0B801CE010E94681EA1
:1006F000882309F444C0B801CE010E941B2288233C
:10070000F1F1B801CE010E942F208823C1F1B80178
:10071000CE010E947721882391F1B801CE010E9479
:100720007F1C882361F1F8018281882309F1CB3590
:100730008DE5D807C1F050F4C115FCE5DF0781F065
:10074000CF3DDC45A9F40E94000F19C0CC35EDE582
:10075000DE0761F0CD35DD4559F40E94430E08C037
:100760000E9456030CC00E944C0E02C00E944F0E05
:10077000C801DF91CF911F910F910C94FF0280E08F
:10078000DF91CF911F910F9108950E94B22380E0D5
:100790000E94201F0E94E7030C94FC1A0E948C1DEB
:1007A0000E94EA030E94C81B0C94B82308950C947D
:1007B000D60381E008950C94D9030895CF93C82FF0
:1007C0000E94D7038C2F0E94DB03CF91089580E015
:1007D0000C94DE030E9477220C94DE030E947722A1
:1007E0009091C001891721F08093C0010C94DE0321
:1007F0000895CF93DF93CDB7DEB72B970FB6F8945C
:10080000DEBF0FBECDBF4F83588769877A878B873E
:1008100061110E948F0D9E012F5F3F4F86E0F9010D
:1008200011928A95E9F785E0FE013796D90101908A
:100830000D928A95E1F789819A814C815D81452BE2
:1008400031F09F3F31F491E08F3F19F403C091E004
:1008500001C090E090FF09C049815A816B817C8181
:100860008D819E810E94B00C05C0C9010E94440385
:100870008111F2CF2B960FB6F894DEBF0FBECDBF1D
:10088000DF91CF910895FC01808191810E940B0A34
:100890000895CF93882309F4A4C0C82F8238C1F4E7
:1008A0000E94772281FD9DC069E3809102019091B1
:1008B00003010E946D230E94B10D2FEF81EE94E0A1
:1008C000215080409040E1F700C0000069E319C06A
:1008D000833801F50E94772280FD83C063E5809113
:1008E0000201909103010E946D230E94B10D2FEF30
:1008F00081EE94E0215080409040E1F700C000007C
:1009000063E580910201909103010E947823CF91C9
:100910000C94B10D8438C1F40E94772282FD61C02D
:1009200067E480910201909103010E946D230E946F
:10093000B10D2FEF81EE94E0215080409040E1F71F
:1009400000C0000067E4DDCF8CEF8C0F813AD0F45B
:100950006C2F80910201909103010E94ED22882367
:1009600049F06C2F80910201909103010E9478233D
:100970000E94B10D6C2F80910201909103010E94A1
:100980006D23C5CF80E28C0F883048F4C77081E0BA
:1009900001C0880FCA95EAF70E94720DB8CFEBE547
:1009A000EC0FE33040F4F0E0E45AFE4F808190E039
:1009B000CF910C94AB22E8E5EC0FE73150F4F0E076
:1009C000EE0FFF1FE25DFE4F80819181CF910C946D
:1009D000C122CD3E30F08C2F0E940F14CF910C9489
:1009E000E114CF910895882309F464C0823879F422
:1009F0000E94772281FF5EC069E38091020190919D
:100A000003010E946D230E94B10D69E310C0833879
:100A1000B1F40E94772280FF4DC063E5809102010E
:100A2000909103010E946D230E94B10D63E58091B6
:100A30000201909103010E9478230C94B10D843837
:100A400079F40E94772282FF35C067E48091020129
:100A5000909103010E946D230E94B10D67E4E7CFDE
:100A60009CEF980F913A10F4682FE1CF90E2980F25
:100A7000983050F4877091E001C0990F8A95EAF799
:100A8000892F0E94780DD9CF9BE5980F933020F4E1
:100A900080E090E00C94AB2298E5980F973120F419
:100AA00080E090E00C94C1228D3E20F00E946A14F8
:100AB0000C94E11408951F93CF93DF93182FEB014B
:100AC0000E944904209741F08FE99FE00197F1F7D8
:100AD00000C000002197F6CF812FDF91CF911F91A9
:100AE0000C94F304893319F060E070E002C060E513
:100AF00070E00C945B05882321F00E94720D0C9429
:100B0000B10D0895882321F00E94780D0C94B10D49
:100B10000895CF92DF92EF92FF920F931F93CF939E
:100B2000DF937C01D62FC72FFC011281058102952E
:100B30000F700E94680D8823B9F01123A9F08C2F43
:100B4000807F803421F080E28D0F883068F08091C2
:100B5000B60282FD09C082E00E94110E0E94680D5B
:100B600091E0D82ED92601C0D12CCC2EC2948FE092
:100B7000C8228C2D90E08C30910508F0CFC1FC018B
:100B8000EA5AFF4F0C94DC2B8C2F807FCF70882388
:100B900011F0C295C07F112399F0CC2309F4AAC1AA
:100BA00080E28D0F883010F0D11104C08C2F0E948C
:100BB000720D03C08C2F0E94820D0E94B10D9AC14C
:100BC0008D2F0E94F304CC2309F4A8C180E28D0F7D
:100BD000883038F1DD2329F18C2F0E94880D24C044
:100BE0008C2F807FCF70803211F0C295C07FDD23C3
:100BF00019F0D130A1F13DC08091B60282FF17C03B
:100C0000112349F0CC2329F08C2F0E94720D0E94F1
:100C1000B10D80E070C180E00E94F304CC2309F4A0
:100C20007DC18C2F0E94780D0E94B10D77C11123D8
:100C300071F0002341F0013031F40E94920D8C2BB1
:100C40000E949A0D6BC10E94920D8C2B1DC0002337
:100C500019F0013009F462C10E94A70D25C01123CB
:100C600021F0063008F05AC10EC0053008F056C118
:100C70001BC0112361F0002331F0F701858180FF53
:100C800039C18F7085838C2F0E947B0547C100235B
:100C900059F0D93309F03FC1FFEF07EE13E0F150EF
:100CA00000401040E1F735C18C2F0E94820536C10B
:100CB0008C2F86958695837019F0813061F02EC156
:100CC000112321F08D2F9C2F937002C080E090E0C3
:100CD0000E94AB222BC1112321F08D2F9C2F9370EA
:100CE00002C080E090E00E94C12220C18D2F11231C
:100CF00019F00E940F1402C00E946A140E94E114AD
:100D000015C18C2F837009F047C011110BC12D2F15
:100D1000229526952770220F220F6D2F6F70862F38
:100D200090E0A0E0B0E0022E04C0880F991FAA1F37
:100D3000BB1F0A94D2F7D4FF10C04FE050E060E030
:100D400070E004C0440F551F661F771F2A95D2F725
:100D5000409550956095709503C040E050E0BA0111
:100D6000C695C695C3708A019B01082B192B2A2BA7
:100D70003B2BC901B801C23049F058F4C13019F019
:100D80000E948A08CFC00E947808CCC00E949C08AC
:100D9000C9C00E947608C6C0112319F08C2F81703B
:100DA00001C08695882309F4BDC02D2F2295269574
:100DB0002770220F220F6D2F6F70862F90E0A0E01A
:100DC000B0E0022E04C0880F991FAA1FBB1F0A940F
:100DD000D2F7D4FF10C04FE050E060E070E004C0F4
:100DE000440F551F661F771F2A95D2F740955095DF
:100DF0006095709503C040E050E0BA01C695C69575
:100E0000C3708A019B01082B192B2A2B3B2BC9018C
:100E1000B801C23049F058F4C13019F00E944F09AE
:100E200081C00E943D097EC00E9461097BC00E9472
:100E3000B00878C0CF70112339F08C2F0E94D608EB
:100E40008D2F0E947B056EC08D2F0E9482058C2FF6
:100E50000E94F70867C0D23F21F128F4D03F41F04B
:100E6000D13FC1F043C0D33F19F1D43F79F03EC028
:100E7000112341F0053008F051C08C2F8F710E9472
:100E80001C094CC0063008F049C0F7CF8091B6026B
:100E900082FF18C0112339F08C2F8F710E94D60861
:100EA0003DC01123C9F38C2F8F710E94F70836C003
:100EB000112329F08C2F8F710E94C1082FC00E942E
:100EC000BC082CC0112349F0CF718C2F0E94D6088A
:100ED00063E08C2F0E94F60D21C081E00E94110E6C
:100EE0000230E0F082E00E94110E18C0112331F0B0
:100EF000002391F28D2F0E94490410C0002399F223
:100F0000D93349F41FEF27EE33E011502040304031
:100F1000E1F700C000008D2F0E94F30488EF8C0DD4
:100F2000843020F40E9477220E94DE03DD20C9F085
:100F30000E94640D80FD15C0F70112820E945E0DB3
:100F40000E94D608C7010E94D2070E945E0DDF9161
:100F5000CF911F910F91FF90EF90DF90CF900C9465
:100F6000F708DF91CF911F910F91FF90EF90DF90E5
:100F7000CF9008950F931F93CF93DF93EC01688177
:100F800079818A810E94160A8C010E9473090E944D
:100F90006408B801CE010E948905DF91CF911F91AD
:100FA0000F910895CF93DF93EC01988189812B8174
:100FB0003C81232B31F08F3F31F481E09F3F19F4C6
:100FC00003C081E001C080E080FD1DC0CE010E9411
:100FD0006503811110C00E94680D8823A1F08A81E9
:100FE000882389F08091B60282FD0DC082E0DF91F6
:100FF000CF910C94110ECE010E94BA07CE01DF9161
:10100000CF910C944603DF91CF91089580E090E05A
:101010000E94AB2280E090E00E94C1220E948F0DCE
:101020000E94B10D0E9412160C94E11480910201ED
:10103000909103010E9483230C9406080E947F0D67
:101040000C94160892959F70963079F010F4925097
:1010500001C09A50923068F4803F69F018F4883EDD
:1010600040F409C0843F29F406C0883E20F0813F47
:1010700011F080E0089581E00895FC018081918164
:101080000E940B0A0E9422080895CF93DF9300D09C
:1010900000D01F92CDB7DEB70F900F900F900F903A
:1010A0000F90DF91CF910895CF93DF9300D000D0C0
:1010B00000D0CDB7DEB726960FB6F894DEBF0FBED0
:1010C000CDBFDF91CF910895089508950C946508E0
:1010D0000C9466080E9468086093D5017093D6014D
:1010E0008093D7019093D8010C9406080C946A0859
:1010F0000F931F930091D5011091D6012091D70134
:101100003091D801602B712B822B932B1F910F9163
:101110000C946A080F931F930091D5011091D6018A
:101120002091D7013091D80160237123822393232A
:101130001F910F910C946A080F931F930091D50192
:101140001091D6012091D7013091D80160277127E5
:10115000822793271F910F910C946A080C946508BD
:101160000E94AE086093D1017093D2018093D301A5
:101170009093D4010C94060860E070E0CB010C94CD
:10118000B0080F931F9341E050E060E070E08A01E7
:101190009B0104C0000F111F221F331F8A95D2F735
:1011A000C901B8011F910F910C94B0080F931F93C0
:1011B00041E050E060E070E004C0440F551F661F3E
:1011C000771F8A95D2F78091D1019091D201A09199
:1011D000D301B091D4018A019B01082B192B2A2B32
:1011E0003B2BC901B8011F910F910C94B0080F93CC
:1011F0001F9341E050E060E070E004C0440F551FD1
:10120000661F771F8A95D2F7409550956095709527
:101210008091D1019091D201A091D301B091D401DC
:101220008A019B01082319232A233B23C901B80102
:101230001F910F910C94B0080F931F9341E050E061
:1012400060E070E004C0440F551F661F771F8A9549
:10125000D2F78091D1019091D201A091D301B091A8
:10126000D4018A019B01082719272A273B27C90196
:10127000B8011F910F910C94B0080F931F93009128
:10128000D1011091D2012091D3013091D401602B72
:10129000712B822B932B1F910F910C94B0080F93FD
:1012A0001F930091D1011091D2012091D30130916F
:1012B000D40160237123822393231F910F910C94F7
:1012C000B0080F931F930091D1011091D20120918A
:1012D000D3013091D40160277127822793271F9172
:1012E0000F910C94B0080895990F990F890FE82F6A
:1012F000E695E695E695877051E001C0550F8A9511
:10130000EAF785E0E89FF0011124EE53FE4F20E05C
:1013100030E070E04081CB01022E02C096958795A7
:101320000A94E2F78170819584278523842781932D
:101330002F5F3F4F2530310569F70895990F990FB9
:10134000890F682F669566956695982F977085E04A
:10135000689FB001112440E050E080E0FB01E40F01
:10136000F51FEE53FE4F208130E0092E02C0369566
:1013700027950A94E2F721703327042E01C0220F2B
:101380000A94EAF7822B4F5F5F4F4530510531F7E2
:101390000895BF92CF92DF92EF92FF920F931F9327
:1013A000CF93DF938C01C090D101D090D201E09017
:1013B000D301F090D4018091D5019091D601A091F4
:1013C000D701B091D801C82AD92AEA2AFB2ACFE14D
:1013D000D0E0D701C6010C2E04C0B695A79597950D
:1013E00087950A94D2F780FD04C0219790F7B12C1D
:1013F00007C0BC2EB8018C2F0E9413110197A9F3CE
:101400008B2DDF91CF911F910F91FF90EF90DF9087
:10141000CF90BF900895CF93DF93EC010E94C9094C
:10142000BE010E941311DF91CF9108951F93CF93B6
:10143000DF93EB019091C101992321F0CB010E9430
:101440000B0A13C0882349F0CB010E94C909182F49
:10145000682FCE010E94740904C0CB010E949E092E
:10146000182FBE01812F0E941311DF91CF911F9180
:1014700008951F93CF93DF93C091D90116E0809117
:10148000DA01C81799F0D0E01C9FF0011D9FF00D04
:101490001124E552FE4F4081518162817381848124
:1014A00095810E9454082196C770E9CFDF91CF91B2
:1014B0001F91089540910B0250910C0260910D0212
:1014C00070910E0280910F02909110020C945408BA
:1014D000EF92FF920F931F93CF93DF9380911002AF
:1014E00082958F7009F065C080910D02882309F400
:1014F00060C08091D901F090DA0110910B02009147
:101500000C0260910E0270910F0291E01F3F09F0F2
:1015100090E0C0910001D0910101292F96E0E92EC1
:101520008F1509F446C06115710521F00F3F21F0B8
:1015300030E003C031E001C0322F90E030FD36C012
:10154000E89EF001E99EF00D1124DF01A552BE4F87
:1015500011963C911197301329C03C91311326C04C
:1015600012963C911297311121C013964D915C91C6
:101570001497461B570B4C175D07C0F4809110025F
:101580008F70806180931002E052FE4F80818F70D7
:10159000806180838BE092E00E94D207DF91CF913F
:1015A0001F910F91FF90EF900C94390A019687706C
:1015B000B7CFDF91CF911F910F91FF90EF900895DA
:1015C0009F92AF92BF92CF92DF92EF92FF920F93D2
:1015D0001F93CF93DF93CDB7DEB761970FB6F89423
:1015E000DEBF0FBECDBF8C0185E0F801DE011D9688
:1015F00001900D928A95E1F7D8011296EC909091A6
:101600000B02E0910C0220910E0230910F02211585
:10161000310531F0EF3F31F481E09F3F19F403C011
:1016200081E001C080E0B82FB1709B2E80FD47C1E2
:10163000D8014C9111965C9111971396AD90BC9086
:1016400014978BE0C82E82E0D82EF0900D02B501E1
:10165000621B730B2091000130910101FF2009F4FE
:10166000D9C0809110026217730708F095C0282F27
:10167000207F09F052C05E1313C0491311C0FE2C25
:10168000E1100EC08F708061809310020E945A0A90
:10169000C6010E94D20780911002F80185834DC1D6
:1016A000AB2831F05F3F31F481E04F3F19F403C0C4
:1016B00081E001C080E080FD03C081E08E2502C092
:1016C00080E090E0F82FF170FF2E80FF1CC0809129
:1016D000D9012091DA0136E0821709F40BC190E0BC
:1016E000389FF001399FF00D1124E552FE4F6181C2
:1016F000561306C06081461303C06281E61203C020
:1017000001968770E9CFFE2CEE2009F416C1809176
:10171000100281608093100254C05E1306C049130A
:1017200004C0E11002C0F80199C0C8010E943D0840
:10173000882361F1EE2051F120911002822F8295D1
:101740008F7090E0029774F080910B0290910C02E0
:1017500098878F831986BB86AA862C87CE01079629
:101760000E94D20786E0F801ABE0B2E001900D9252
:101770008A95E1F70E94680A0E945A0A0AC05E1719
:1017800011F1C8010E943D0881112CC0C8010E94BE
:10179000D207FF24F394D1C0282F207F81F77A2D20
:1017A000B98AA88A6E2D89890E9445088BE092E04B
:1017B0000E94D20786E0D6011D928A95E9F70E9421
:1017C0005A0AF12CBAC04913DCCFE110DACFF80184
:1017D0008583C8010E94D20786E0D6011D928A95B2
:1017E000E9F7ABC0EE2091F220911002822F829592
:1017F0008F7090E002970CF4B5CF80910B0290911E
:101800000C029A8389831B82BD82AC822E83CE0117
:101810000196A6CF6217730708F044C0FE2CEE2095
:1018200009F4B4CF5E1330C049132EC020911002CA
:1018300020FD21C0822F82958F70482F50E04115E6
:101840005105C9F0F80125834F30510541F08F5FF4
:10185000982F9295907F822F8F70892B8583C80156
:101860000E94D20786E0F801ABE0B2E001900D9251
:101870008A95E1F73CC086E0F801ABE0B2E0019068
:101880000D928A95E1F759C0C8010E943D08811167
:1018900069CF80911002816080931002C8010E947C
:1018A000D2074BC07A2DB98AA88A6E2D89890E94E9
:1018B000450886E0D6011D928A95E9F718C0EE200A
:1018C00009F464CFC8010E943D08F82E882309F46A
:1018D0005DCF86E0F801ABE0B2E001900D928A9511
:1018E000E1F78BE092E00E9443040E94680A0E94A4
:1018F0005A0A23C04D875E878D859E850E940B0AFC
:10190000292F22952F70223028F49F7039F08111F1
:1019100005C00BC0243028F49F7049F4805E8830E5
:1019200020F0C8010E94D2079F2CF92C06C0D801D4
:1019300015969C91907F91F7F8CF8F2D61960FB6F9
:10194000F894DEBF0FBECDBFDF91CF911F910F91F5
:10195000FF90EF90DF90CF90BF90AF909F90089551
:101960001F93CF93DF93CDB7DEB72C970FB6F894C4
:10197000DEBF0FBECDBF4F83588769877A878B87BD
:101980009C87CE0107960E94E00A8823D1F09F81B0
:1019900088852A853B85232B31F08F3F31F481E008
:1019A0009F3F19F403C081E001C080E080FD47C083
:1019B0004F81588569857A858B859C850E9454085E
:1019C0003EC086E0FE013796DE01119601900D9231
:1019D0008A95E1F7FF81E8856A857B856115710548
:1019E00031F0EF3F31F481E0FF3F19F403C081E0B3
:1019F00001C080E080FD23C02091DA0130E0C90100
:101A00000196877099274091D90150E08417950776
:101A1000F1F1F983EA837D836C8396E0929FD00194
:101A2000939FB00D1124A552BE4FFE013196019037
:101A30000D929A95E1F78093DA010E94390A16E037
:101A40008091D9019091DA01891771F1189FC00135
:101A5000112485529E4F0E94E00A882329F1E091CB
:101A6000D9011E9FF0011124E552FE4F40815181A2
:101A700062817381848195810E9454088091D9018B
:101A800090E00196877099278093D901D9CF0E9461
:101A90001E081092DA011092D901EBE0F2E086E024
:101AA000DF011D928A95E9F72C960FB6F894DEBFF8
:101AB0000FBECDBFDF91CF911F910895809131026C
:101AC0008595859585950895809131028770089553
:101AD00090913102977081E009F480E0089580913F
:101AE0005402089590915402892B809354020895D2
:101AF0008095909154028923809354020895109206
:101B00005402089590915302892B809353020895B3
:101B100080959091530289238093530208951092E7
:101B20005302089580913202089508950C94950D02
:101B30000C94960D9091B60292FD08C090913202DD
:101B4000981721F0809332020C94980D089580919B
:101B50003202882329F01092320280E00C94980D12
:101B60000895CF93DF93E0910201F09103018091FA
:101B700054028083E0910201F091030190818091F1
:101B80005302892B808380913202882381F0E09177
:101B90000201F09103019081892B808380910201E1
:101BA000909103010E94D72281110E94A70DC0913C
:101BB0000201D091030140E250E061E172E0CE0108
:101BC0000E94202C892B69F080E2FE01A1E1B2E0A5
:101BD00001900D928A95E1F7CE01DF91CF910C949F
:101BE0008322DF91CF9108950C94950D9091B602C8
:101BF00092FD10C098E0899F90011124262B20931C
:101C000031020E94D608809131028595859585958F
:101C10000C94F40D0C94D6081092310280E00C94D0
:101C2000F40D209131028095822380933102982F08
:101C3000977099F430E0482F082E000C550B2417AC
:101C4000350759F09091B60292FD07C085958595AC
:101C500085950E94F7080C940C0E08959091B60299
:101C600092FB222720F9281769F080FB92F99093C4
:101C7000B6028091B5029091B6020E947C0E82E07D
:101C80000C94110E08958091B60282FB882780F98A
:101C900091E089270C942E0E81E00C942E0E80E0AA
:101CA0000C942E0E6FEF7FEF80E090E00C945F2C91
:101CB00080E090E00E943B2C21E0893E9E4F09F09D
:101CC00020E0822F089582E090E00C942D2C83E098
:101CD00090E00C942D2CCF9384E090E00E942D2C6A
:101CE000C82F82E290E00E942D2C2C2F30E0A90119
:101CF000582BCA01CF910895CF93C92F682F84E044
:101D000090E00E94412C6C2F82E290E0CF910C94E5
:101D1000412CAB01BC018FE090E00C94532CAB0143
:101D2000BC0183E190E00C94532C60E070E0CB01A7
:101D30000C948F0E60E070E0CB010E94890E0C9431
:101D4000950E69EE7EEF80E090E00E945F2C60E0EF
:101D500082E090E00E94412C60E083E090E00E94ED
:101D6000412C1092D5011092D6011092D7011092F9
:101D7000D80160E084E090E00E94412C60E082E2C3
:101D800090E00E94412C60E085E090E00E94412CB0
:101D900060E086E090E00E94412C6FEF87E090E0E9
:101DA0000E94412C40E050E0BA0188E090E00E949F
:101DB000532C60E08DE090E00E94412C40E050E028
:101DC000BA0188E190E00E94532C60E087E190E046
:101DD0000E94412C40E050E0BA018CE190E00E946A
:101DE000532C60E070E080E290E00E945F2C40E0C5
:101DF00050E0BA0188E190E00E94532C0C949A0EB6
:101E00000C94A10E682F8EE090E00C94412C0E945F
:101E10003C2460935E0270935F0280936002909313
:101E2000610260935A0270935B0280935C0290930C
:101E30005D02089585B7806885BF85B7806885BFD6
:101E4000089581E008950C94210F08950C94250FB6
:101E50000C94250F0C94280F0C94250F0C942C0F28
:101E60000C94250F0E941A0F8FEE91E10E946D22B3
:101E70000E94300F0C942E0F0E94260F0C94250FF9
:101E80000E9409120E94DD030C94EE1F0E94272479
:101E90000E94E5120E94400F0E948C1D0E948D1B23
:101EA000E5EBF2E08081806880838091B5029091BB
:101EB000B6020E947C0E0C942A0F8F929F92AF92D2
:101EC000BF92CF92DF92EF92FF920F931F93CF9327
:101ED000DF93CDB7DEB72A970FB6F894DEBF0FBEFB
:101EE000CDBF0E94FA12982E81110E94070F85E53E
:101EF000A82E82E0B82E00E010E0802E802F0E94F5
:101F00002D12D82EF501C1905F01C826B1F40F5FE4
:101F10001F4F0530110589F78FEF89838A831B8254
:101F20000E9430248160782F9D838C8349815A815F
:101F30006B818D810E94F9032FC08091620281FD27
:101F40000E943312E12CFF24F3948C2D8F21F1F0A9
:101F50000E94230F882399F0EE828F82DF2081E098
:101F600009F480E088870E9430248160782F9A8766
:101F700089874E815F8168858A850E94F903F8010F
:101F8000EB5AFD4F8081F826F08206C0E394FF0CE7
:101F9000F4E0EF12DACFBBCF81E0911001C080E016
:101FA0002A960FB6F894DEBF0FBECDBFDF91CF915A
:101FB0001F910F91FF90EF90DF90CF90BF90AF9067
:101FC0009F908F9008950E945D0F0E94D11B0E94E8
:101FD000521F0E94FF140C94EE03CF93DF930E94D4
:101FE0001811EC01811521E5920708F045C0811513
:101FF00030E5930708F094C0883E910528F5803EAF
:10200000910508F0F8C0883A910570F4853A910579
:1020100008F07CC08130910509F475C008F4E8C06F
:10202000049708F0E8C0E4C08F3B910508F0E0C0D9
:10203000C85AD0E0CC0FDD1FC15ADE4F0990D881BD
:10204000C02DCE019464D8C0811540E2940758F4A5
:10205000811551E0950708F0CEC08D3E910508F43A
:10206000C7C09065C9C0C11580E4D80708F4C0C0D6
:10207000DF70CE01906AC0C0811525E59207A8F4F3
:10208000811534E5930708F095C0811543E5940761
:1020900008F07BC0811552E5950708F061C0D82F84
:1020A000CC27CE01816F906AA7C0C11589E5D807FA
:1020B000A0F4C11528E5D20708F082C0C11536E5A5
:1020C000D30708F095C08C2F0E94AC118F7190E05F
:1020D000D82FCC27CE0190628FC0C1154AE5D40716
:1020E00008F474C0CE0190568115904208F080C06B
:1020F0008D2F8F710E94AC11DD27D0628F71AE01E0
:10210000582BCA0179C081E090E076C0C55AD0E072
:10211000C357DE4F8881C82FD0E0CE0190646CC0D9
:1021200074E0969587957A95E1F7282F23703C2FD8
:10213000337081E090E002C0880F991F3A95E2F772
:102140009C68AC01522B9A019C2F9F709695969596
:1021500050E2959FE0011124C9018C2B9D2B4CC0AE
:102160008370992721E030E002C0220F331F8A9547
:10217000E2F79C2F9695969580E2989FE0011124B6
:10218000C22BD32BCE019C6837C08370992721E0E6
:1021900030E002C0220F331F8A95E2F79C2F9695FC
:1021A000969540E2949FE0011124C22BD32BCE01DF
:1021B0009A6822C0D82FCC27CE01846F906A1CC0A9
:1021C000DC2FCC27CE01806F906A16C08C2F8F70C9
:1021D0000E94AC1194E0D695C7959A95E1F7CF701F
:1021E000D0E0DC2FCC27D0699E01282BC90104C088
:1021F00080E090E001C0CE01DF91CF910895E72FFC
:10220000F0E095E0899FE00DF11D1124EE0FFF1F16
:10221000EE0FFF1FE60FF11DEE0FFF1FEA51FF4FFC
:102220008591949108950E94FF100E94ED0F0895EA
:102230008238910569F1B0F48133910509F46DC0DC
:1022400048F48932910509F463C08A32910509F492
:1022500069C008958533910509F455C08933910506
:10226000B9F00895833E910569F138F4803E9105F7
:10227000B1F0823E910509F10895863E9105A9F1DC
:10228000873E9105B9F1843E910509F064C023C0F1
:102290002091B50220FD4FC021FD4DC008958091D1
:1022A000B50280FD44C08091B60280FF44C0809199
:1022B000B50284FD42C083EE4DC08091B50282FF1D
:1022C00038C0F5CF8091B50282FD33C08091B6024F
:1022D00080FD31C0ECCF8091B60281FF32C0809189
:1022E000B50284FD2AC087EE35C08091B50283FF18
:1022F00026C0F5CF8091B50283FD21C08091B60242
:1023000081FD1FC0ECCF8091B50285FD1CC01DC0B2
:102310008091B50285FD19C016C08091B50286FD79
:1023200016C017C08091B50286FD13C010C089E3A6
:1023300011C082EE0FC080EE0DC080E00BC086EEB3
:1023400009C084EE07C089E205C085E303C08AE2C4
:1023500001C081E390E008959091B50292FF0DC015
:10236000282F2871283019F4877F846006C0282F11
:102370002471243011F48B7F886093FF0DC0282FC7
:102380002871283119F4877E846106C0282F2471B2
:10239000243111F48B7E88612091B60220FF0DC09C
:1023A000382F3871383019F4877F816006C0382F94
:1023B0003171313011F48E7F886021FF0DC0282FDC
:1023C0002871283119F4877E816106C0282F217178
:1023D000213111F48E7E886194FD877E089580E01E
:1023E00008950C94520E0E94FA128FE39CE9019713
:1023F000F1F700C000000E94FA1280E00E942D1246
:1024000080FF04C00E94F1110C947D2408950C9467
:10241000F3110E94580E811102C00E94000F0E9409
:10242000630E809362020E946B0E9093B6028093BB
:10243000B5020E9407120E94670E682F70E080E0CC
:1024400090E00E9476086091D1017091D201809154
:10245000D3019091D4010C94AE08E82FF0E0E4543D
:10246000FD4F80810895089580EA8A95F1F70895D7
:1024700000C008950C94341208950C943C120C94EE
:102480003D120C943C120C944112F894E82FE29502
:10249000EF70F0E031A1282F2F7081E090E001C0B3
:1024A000880F2A95EAF7982F9095932391A392A1EC
:1024B000892B82A3789408950F931F93CF93DF9372
:1024C000C0E9D1E089918F3F11F00E94451281E06F
:1024D000C439D807B9F7C4E9D1E009E911E0899115
:1024E0008F3F11F00E9445120C171D07C1F7DF91B5
:1024F000CF911F910F910895EF92FF920F931F9329
:10250000CF93DF93C62FD0E0C057DE4F28812F3FF7
:1025100009F454C0042F162F7C01F894E22FE295A1
:10252000EF70F0E081A1422F4F7021E030E001C058
:10253000220F4A95EAF7822B81A382A120952823B6
:1025400022A378940E94381264E971E0F701A70190
:102550004B5F5F4FF12C302F3095DB012D91BD018A
:102560002F3FB1F0822F82958F7090E0DC01909622
:102570008C9190E02F7002C0959587952A95E2F78F
:1025800080FD06C08081802B8083FF24F39403C0EC
:102590008081832380833196E417F507F1F68881E3
:1025A0008F3F11F00E9445126F2D812FDF91CF9147
:1025B0001F910F91FF90EF900C943A12DF91CF9101
:1025C0001F910F91FF90EF9008950E945C1285E09B
:1025D000ECEBF2E0DF01982F1D929A95E9F7E7EB1B
:1025E000F2E0DF011D928A95E9F785E00E9447132A
:1025F0000C945103EF92FF920F931F93CF93DF93AD
:1026000000D000D01F92CDB7DEB78E010F5F1F4FF5
:1026100085E0F80111928A95E9F7F12CEE24E39414
:102620004E2D6F2DC8010E947C12F394EE0CF4E045
:10263000FF12F6CF45E050E0B80187EB92E00E9430
:10264000202CFF24F394009709F4F12C892B41F0FE
:1026500085E0F801A7EBB2E001900D928A95E1F7D1
:102660002F2D45E06CEB72E087EB92E00E9448135F
:102670000E9453038F2D0F900F900F900F900F908B
:10268000DF91CF911F910F91FF90EF9008950895E2
:10269000FF920F931F93CF93DF938C01F62ED72FCA
:1026A000C42F222349F081E0809365020E943024E8
:1026B0009093640280936302809165028823C1F045
:1026C00080916302909164020E944824059780F0F3
:1026D000EF2DFD2FD8014C2F50E0CD01801B910B29
:1026E000841795071CF48D918193F7CF10926502A2
:1026F000DF91CF911F910F91FF9008950E9448267E
:102700000E94460F0C9454260E9458260E94E30F04
:102710000C9472260E94CE230E942F260E94320F14
:102720000E947E130E9484130E943C0FFBCF809175
:102730006C0280FF06C06091090170E0660F771F90
:1027400026C081FF04C06091090184E005C082FFBA
:1027500007C06091090188E0689FB001112417C08B
:1027600090916B029923D1F060910801961788F738
:102770002091090188E0289F90011124929FA001D7
:10278000939F500D112470E0CA010E94A62B60385F
:10279000710540F46115710519F406C068E070E038
:1027A000862F08958FE7089581E0089580916C0247
:1027B00080FF08C06091050170E07595679575957B
:1027C000679521C081FF06C06091050170E0759595
:1027D000679519C082FF04C06091050170E010C0C8
:1027E00090916A02992399F0609104019617A0F7DD
:1027F00080910501899FC001112470E00E94A62BE1
:102800006038710540F46115710519F406C061E086
:1028100070E0862F08958FE7089581E008958D3E3A
:1028200021F40E949713819504C08E3E29F40E94E2
:1028300097138093700208958F3E21F40E9497139E
:10284000819504C0803F29F40E94971380936F0202
:102850000895893F19F40E94D61305C08A3F31F4C8
:102860000E94D61381958093710208958B3F21F4C5
:102870000E94D613819504C08C3F29F40E94D61380
:102880008093720208959FE0980F983078F421E0C9
:1028900030E0A90102C0440F551F9A95E2F7CA0122
:1028A00090916E02892B80936E0208958D3F21F4E2
:1028B00080916C0281600BC08E3F21F480916C028C
:1028C000826005C08F3F29F480916C028460809300
:1028D0006C0208958D3E39F49091700297FF35C0D7
:1028E0001092700259C08E3E29F490917002191610
:1028F000BCF32BC090916F028F3E29F497FF25C047
:1029000010926F0249C0803F19F41916CCF31DC014
:1029100090917102893F29F41916BCF4109271024A
:102920003BC08A3F19F497FF10C0F8CF8B3F39F4B2
:102930009091720297FF09C0109272022DC08C3FD5
:1029400021F4909172021916BCF39FE0980F983011
:1029500080F421E030E0A90102C0440F551F9A9590
:10296000E2F7CA01809590916E02892380936E02EE
:1029700013C08D3F21F480916C028E7F0BC08E3F7F
:1029800021F480916C028D7F05C08F3F29F48091E6
:102990006C028B7F80936C0280916F02811106C064
:1029A00080917002811102C010926B0280917102BD
:1029B000811106C080917202811102C010926A02D8
:1029C00008950E94302420916F02211104C02091AB
:1029D0007002222321F09093690280936802209173
:1029E0007102211104C020917202222321F09093E0
:1029F0006702809366028DE692E00C949D22EF922E
:102A0000FF920F931F93CF93DF9300D000D000D09D
:102A1000CDB7DEB786E0EDE6F2E0DE01119601907B
:102A20000D928A95E1F7E0906F02F09070020091AC
:102A300071021091720210926F0210927002109245
:102A4000710210927202E11003C0FF2009F45DC010
:102A500080916802909169020E944824AC01909193
:102A60006B02992339F020910A0130E024173507D1
:102A700058F04BC020910B018AE0289F900111244F
:102A80002417350718F041C09F3F19F09F5F9093BE
:102A90006B02EE2061F00E9497131E1414F09FEF5A
:102AA00001C091E0989F902D112490936F02FF2018
:102AB00061F00E9497131F1414F09FEF01C091E082
:102AC000989F902D11249093700230916F023323C0
:102AD000E1F0209170022223C1F045EB3403C001E4
:102AE0001124992319F090936F0203C081E0809321
:102AF0006F0235EB2303C0011124992319F0909341
:102B0000700203C081E080937002011103C01123A1
:102B100009F45DC080916602909167020E9448248A
:102B2000AC0190916A02992339F02091060130E0BE
:102B30002417350758F04BC0209107018AE0289FE1
:102B4000900111242417350718F041C09F3F19F058
:102B50009F5F90936A02002361F00E94D6131016C3
:102B600014F09FEF01C091E0989F902D1124909355
:102B70007102112361F00E94D613111614F09FEF19
:102B800001C091E0989F902D112490937202309192
:102B900071023323E1F0209172022223C1F045EB50
:102BA0003403C0011124992319F09093710203C0DA
:102BB00081E08093710235EB2303C0011124992336
:102BC00019F09093720203C081E0809372028091A9
:102BD0006F0281110BC080917002811107C080913A
:102BE0007102811103C08091720281110E94E1146F
:102BF000EB82FC820D831E8386E0FE013196ADE6FA
:102C0000B2E001900D928A95E1F726960FB6F894FE
:102C1000DEBF0FBECDBFDF91CF911F910F91FF900F
:102C2000EF900895EDE6F2E086E0DF011D928A95CF
:102C3000E9F710926B0210926A0210926C020895EA
:102C4000EF92FF920F931F93CF93DF938B01682F27
:102C500011110AC0442329F0E82FF0E0E35EFC4F95
:102C60006491762F862F75C0212F30E0E82FF0E099
:102C7000442321F0E35EFC4FE491F0E046E0049F42
:102C8000C0011124CFEFD0E0BE010E94922B4BEA8D
:102C90004603C001479F900D1124800F911D800FA6
:102CA000911D982F990F890FAE01421B530B4E9F18
:102CB000D0014F9FB00D5E9FB00D11249B2F189F28
:102CC000A0011124452F55278E01041B150B0E9FC3
:102CD000A0010F9F500D1E9F500D11247E01E81A78
:102CE000F108E29E8001E39E100DF29E100D11246A
:102CF000212F3327C21BD30BCE9F9001CF9F300DC6
:102D0000DE9F300D112462307105A9F048F4611581
:102D1000710569F061307105C9F48B2F752F0DC0F5
:102D20006430710581F058F06630710579F47E2FBA
:102D30008B2F932F0DC0832F7B2F9E2F09C08E2F9B
:102D40007B2F952F05C08E2F732F02C07E2F852FCE
:102D5000692FDF91CF911F910F91FF90EF90089510
:102D600041E00E942016089508950E94B01608952B
:102D7000CF93DF93762FE901682F842F0E94B51639
:102D8000798368838A83DF91CF9108958091C1020E
:102D9000282F269530E02115310519F481708260C5
:102DA00005C02532310524F0817088648093C1020A
:102DB000089588E090E00C94352CCF92DF92EF924A
:102DC000FF926B017C010E94C616B701A60188E044
:102DD00090E0FF90EF90DF90CF900C94532CE1ECBB
:102DE000F2E083E0808311828FEF828383831482F9
:102DF00060817181828193810C94DD168091C10282
:102E000080FF02C08695089580E008959091C502E4
:102E1000933018F49F5F9093C502882351F060911E
:102E2000C1027091C2028091C3029091C4020C94BD
:102E3000DD16089581E00C9406179091C502992340
:102E400019F091509093C502882351F06091C1020E
:102E50007091C2028091C3029091C4020C94DD165D
:102E6000089581E00C941D1770E00C94042060918B
:102E700010018091C10280FF0AC080910F0123E000
:102E8000829FC00111248A539D4F0C943417809166
:102E9000110190911201891780F7E82FF0E09F014E
:102EA000220F331FE20FF31FEA53FD4F11821082EE
:102EB00012828F5FF0CF9091C10290FF16C0909167
:102EC000110120911201921770F4E92FF0E0DF0157
:102ED000AA0FBB1FEA0FFB1FEA53FD4F81836083DC
:102EE00042839F5FF0CF0C9437170895CF93DF9301
:102EF00000D01F92CDB7DEB79091C10290FF0AC0FB
:102F00009E012F5F3F4F0E94B8164B8169818A81D5
:102F10000E945B170F900F900F90DF91CF91089553
:102F2000CF93DF93EC01EC81F0E0E856FE4F449143
:102F3000E1ECF2E0628181810E9476178C818F5FE3
:102F40008C83DF91CF910895CF93DF93EC01E1EC77
:102F5000F2E0438162818C810E9476178C818F5FC1
:102F60008C83DF91CF9108950F931F93CF93DF93BD
:102F700000D01F92CDB7DEB78C0180917302811112
:102F80000AC09E012F5F3F4F4FEF6FEF0E94B816B0
:102F90008A8180937302F8018481813051F028F096
:102FA000823061F4409173020AC08091730240E064
:102FB00007C06091730240E080E003C040E080E021
:102FC00060E00E945B17F801848190E0019663E065
:102FD00070E00E94A62B84830F900F900F90DF91DA
:102FE000CF911F910F910895AF92BF92CF92DF9230
:102FF000EF92FF920F931F93CF93DF9300D01F9216
:10300000CDB7DEB7182FF62E042FE22E9091C10215
:1030100090FF6DC0E92FE695AE2FB0E0A756BE4FEA
:103020008C9180937F029E7F923061F49E012F5F8E
:103030003F4F812F0E94B8164B8169818A810E947F
:103040005B1743C0823019F40091C4023EC0863041
:1030500019F41091C20239C08930D9F38931A9F528
:10306000E9518E2F8170D82EE695F0E0E856FD4F9D
:10307000A590B490C12CBB2460911301C61618F51D
:103080002C2D30E0A29EC001A39E900DB29E900D0B
:10309000112470E00E94922B812FD11002C0860F64
:1030A00001C0861B90911101290F311DA901440F08
:1030B000551F240F351F2A533D4F402F6F2D0E945F
:1030C000B816C394D9CF0E9437171093C202F0925A
:1030D000C3020093C402EE2051F06091C1027091CE
:1030E000C2028091C3029091C4020E94DD160F902B
:1030F0000F900F90DF91CF911F910F91FF90EF9064
:10310000DF90CF90BF90AF900895E1ECF2E0918115
:10311000282F4381628188E0890F0C94F41781E0A5
:103120000C948518E1ECF2E09181282F43816281B3
:1031300088EF890F0C94F41781E00C949218E1EC5D
:10314000F2E0628128E0620F08F46FEF282F4381DC
:1031500081810C94F41781E00C949F18E1ECF2E06B
:10316000628128E0621B08F460E0282F438181819E
:103170000C94F41781E00C94AE18E1ECF2E043817A
:1031800028E0420F08F44FEF282F628181810C94D0
:10319000F41781E00C94BD18E1ECF2E0438128E0E3
:1031A000421B08F440E0282F628181810C94F417BF
:1031B00081E00C94CC1820E00C94F417FF920F934C
:1031C0001F93CF93DF93EC01F12C0FEF10E0609190
:1031D0001301F616F0F4809111012F2D30E0280F25
:1031E000311DC901880F991F280F391F2A533D4FE0
:1031F00070E0C8010E94A62B962F8C814091C402DA
:103200006091C302F99E800D11240E94B816F394B8
:10321000DECF0E9437179A818C8190FF02C08F5FAA
:1032200001C081508C83DF91CF911F910F91FF904E
:103230000895BF92CF92DF92EF92FF920F931F9368
:10324000CF93DF93FC01828180FF02C00FEF01C0AA
:1032500001E010E080911301181708F040C0809140
:103260001101C12ED12CE601C80FD11DCE01880F4E
:10327000991FC80FD91FCA53DD4F198218821A82AD
:1032800034E0E32EF12CB12C809175028B0D85304A
:1032900014F0837005C087FF03C090911301890F5C
:1032A000082E000C990BC816D90691F48091C4021F
:1032B0008E9DA0018F9D500D1124559547955595D4
:1032C00047959E016091C3028091C2020E94B81688
:1032D000B00EF1E0EF1AF108B9F61F5FBBCF0E9404
:1032E000371780917502013031F4811102C080914D
:1032F0001301815007C090E001966091130170E0C6
:103300000E94A62B80937502DF91CF911F910F91A0
:10331000FF90EF90DF90CF90BF900895CF93809172
:10332000110190911201891770F4E82FF0E09F01CC
:10333000220F331FE20FF31FEA53FD4F1182108259
:1033400012828F5FF0CFC0E060911301C617C0F505
:10335000EC2FF0E070E0CF010E94A62B209111012C
:10336000820F20917402022E000C330B90E0E217C2
:10337000F307CCF020910E01022E000C330B2E1718
:103380003F078CF09C01220F331F820F931F9C017B
:103390002A533D4F4091C4026091C3028091C20202
:1033A0000E94B8160BC0FC01EE0FFF1F8E0F9F1F6F
:1033B000FC01EA53FD4F118210821282CF5FC4CF0D
:1033C0000E94371720910D0180917402820F809323
:1033D000740290910E01920F90930E0119165CF4F5
:1033E000082E000C990B4091130150E041505109F7
:1033F000841795071CF0219520930D01CF91089516
:103400008F929F92AF92BF92CF92DF92EF92FF92F4
:103410000F931F93CF93DF938C01FC014481C42F42
:10342000D0E09E01DE010E94EA2B9B01AC010E94CC
:10343000002C6B017C01E0E2F0E0EC1BFD0BA5E54C
:10344000B0E09B01AC010E94002C4B015C019F018C
:10345000DF010E94E22B9B01AC010E940B2C9B011F
:10346000AC012C0D3D1D4E1D5F1DC501B4010E9418
:10347000BA2BC22FD22F2A3228F4F3E02F9F9001CB
:1034800011240DC025E530E02C1B3109C901880F3E
:10349000991F280F391F37FF02C02F5F3F4F359507
:1034A0002795C22FC095F12C85E5E82EED1A809165
:1034B0001301F816C8F4F1FC02C08E2D01C08D2F47
:1034C000909111012F2D30E0290F311DA901440FDA
:1034D000551F240F351F2A533D4F4C2F6091C302B7
:1034E0000E94B816F394E3CF0E943717F801848145
:1034F000811102C091E003C0803219F49FEF9093D4
:103500000C0190910C01890FF8018483DF91CF9118
:103510001F910F91FF90EF90DF90CF90BF90AF90F1
:103520009F908F9008950F931F93CF93DF93EC019B
:1035300000E010E080911301282F30E002171307FC
:1035400024F5909111019801290F311DA901440F13
:10355000551F240F351F2A533D4F869590E04C810F
:10356000081719071CF4442331F002C0411103C0AD
:103570004091C40201C040E06091C3028091C20248
:103580000E94B8160F5F1F4FD5CF0E9437178C814E
:1035900090E00196817099278C83DF91CF911F91E4
:1035A0000F910895E1ECF2E080818E7F808360814D
:1035B0007181828193810E94DD16109280022FEF2B
:1035C00080E792E0215080409040E1F700C0000089
:1035D0000C943717E1ECF2E080818E7F80831092AB
:1035E00080022FEF80E792E0215080409040E1F789
:1035F00000C000000C9437171092800280917D0269
:1036000081110AC081E080937D028091C1028170A6
:1036100080937C020C94EA1A08956091C102669529
:1036200070E04BE050E084E191E00E94132C892B84
:1036300019F481E0809380020E94302490937702F5
:103640008093760208959091C10290FF35C09170E9
:10365000811102C0926006C0853210F0986402C0E9
:10366000880F982B9093C102662351F06091C1029C
:103670007091C2028091C3029091C4020E94DD1633
:103680006091C102669570E04BE050E084E191E00A
:103690000E94132C892B19F01092800202C00E9404
:1036A0000D1B81E0809379024091C4026091C302B6
:1036B0008091C2020C94DB180895682F9091C1028A
:1036C000969581E0890F853208F081E00C94231BE8
:1036D00081E00C945D1B682F9091C10296958FEF4D
:1036E000890F09F484E20C94231B81E00C946B1B7A
:1036F00061E00C94231BE1ECF2E080818160808327
:1037000086950C94781B8091C10280FD0C94D21A8E
:103710000C947B1B60E00C94231B80917E02811132
:103720002EC00E94580E811104C00E94000F0E94FA
:10373000EF160E94D9166093C1027093C202809363
:10374000C3029093C4026E7F61F40E94EF160E9440
:10375000D9166093C1027093C2028093C302909302
:10376000C4020E94C616109280028091C10280FF9E
:1037700003C086950E948A1B81E080937E02089593
:10378000E1ECF2E080818160808386950C948A1B55
:1037900010927D0280917C0281110E94C01B0C94CA
:1037A0000D1B0F931F93CF93DF938091800288238B
:1037B00009F485C080917F02E091C102E695E81B83
:1037C000E0937802823049F4F0E0EC56FE4FE49149
:1037D000CE2FD0E000E917E149C0863049F4F0E08F
:1037E000EF56FE4FE491CE2FD0E004EA17E13EC041
:1037F000893051F4E695F0E0E257FE4FE491CE2F88
:10380000D0E00EED18E132C08F3051F4E695F0E0D3
:10381000E557FE4FE491CE2FD0E009E119E126C033
:10382000853149F4F0E0E857FE4FE491CE2FD0E027
:103830000EE819E11BC0883181F0833239F4E6E8E3
:10384000F1E0C591D49104EB17E110C0843251F43A
:10385000C4EFD1E003E91AE109C0C8E2D0E000E01A
:103860001AE104C0C0EDD7E004EB16E180917902C3
:10387000882361F0109279020E943024909377029D
:103880008093760210927B0210927A020E9430247A
:10389000E0917602F09177028E1B9F0B8F3F9F473E
:1038A00070F4EC0FFD1FF0937702E093760286E749
:1038B00092E0F801DF91CF911F910F910994DF9170
:1038C000CF911F910F910895882311F0FA0101C043
:1038D000FB010994CF93DF93C82FD62F0E94FE16C9
:1038E0008C1740F00E94FE168D1720F4DF91CF91C7
:1038F0000C94681B8C2FDF91CF910C94781B1F9335
:10390000CF93DF93FB0112811111C3C0EC010E9420
:103910006F0D8272CD3CFCE5DF0709F49AC0A8F573
:10392000C73CECE5DE0709F476C0A8F4C43C9CE58E
:10393000D90709F45FC028F4C33CDC4509F457C03B
:1039400054C0C53C9CE5D90709F459C0C63CDC45C8
:1039500009F45CC04AC0CA3CFCE5DF0709F46AC050
:1039600050F4C83CECE5DE0709F45AC0C93CDC451C
:1039700009F45BC03AC0CB3C9CE5D90709F45FC0B1
:10398000CC3CDC4509F460C030C0C23DFCE5DF073B
:1039900009F46FC088F4CF3C9CE5D90709F460C0F6
:1039A00008F45CC0C03DFCE5DF0709F45CC0C13D24
:1039B000DC4509F45BC019C0C53D9CE5D90709F495
:1039C00060C050F4C33DFCE5DF0709F455C0C43DB9
:1039D000DC4509F454C009C0C63D9CE5D90709F48B
:1039E00055C0CE35DD4509F454C011E052C00E94E7
:1039F000831B4FC045E75BE168E67BE104C048E616
:103A00005BE165E77BE10E94641C43C04CE958E13F
:103A10006FE878E1F8CF4FE858E16CE978E1F3CF4F
:103A20004AEB58E16BEA78E1EECF4BEA58E16AEBFA
:103A300078E1E9CF48ED58E169EC78E1E4CF49EC71
:103A400058E168ED78E1DFCF41E357E16AE177E1E2
:103A5000DACF4AE157E161E377E1D5CF81E017C0E2
:103A600065E082E010C068E086E00DC06EE089E0AD
:103A70000AC064E18FE007C067E185E104C088E126
:103A800006C062E289E10E946A1C03C083E20E94D0
:103A9000781B812FDF91CF911F91089586E090E0F0
:103AA0000C942D2C682F86E090E00C94412C809192
:103AB000D202847089618093D2020C94521D80914D
:103AC000D20286958695869508958091D20281FDD1
:103AD00007C082608093D2020E94521D0C94531F33
:103AE00008958091D20281FF07C08D7F8093D2021A
:103AF0000E94521D0C945F1F08958091D20281FD97
:103B00000C94711D0C94651D8091D2028695817074
:103B1000089580911F0108950E94580E811104C0DC
:103B20000E94000F0E94571D0E944E1D8093D202DA
:103B3000282F26952695269530E02430310524F04F
:103B4000877088618093D2028091D20280FF04C086
:103B500086958695869501C080E00C94201F209163
:103B6000D202822F869586958695482F50E0433065
:103B7000510554F48F5F982F990F990F990F822F49
:103B80008770892B8093D2028091D20281608093CA
:103B9000D2020E94521D8091D2028695869586950A
:103BA0000C94201F8091D202982F96959695969509
:103BB000A1F0915E990F990F990F8770892B8093CF
:103BC000D202887F91E009F490E08091D20290FBCC
:103BD00080F98093D2020E94521D8091D202869574
:103BE000869586950C94201F8091D20280FD13C08B
:103BF00081608093D202813019F489E08093D202EF
:103C00008091D2020E94521D8091D20286958695A3
:103C100086950C94201F08958091D20280FF08C0E1
:103C20008E7F8093D2020E94521D80E00C94201F50
:103C300008958091D20280FD0C940C1E0C94F41D0A
:103C40009091D202892F8695869586958F5F8F7188
:103C50009770843038F4880F880F880F892B8093F1
:103C6000D20202C09093D2028091D202887F91E06A
:103C700009F490E08091D20290FB80F98093D20207
:103C80000E94521D8091D2028695869586950C944D
:103C9000201F843008F083E09091D2029770282F83
:103CA000220F220F220F922B9093D202987F21E0B5
:103CB00009F420E09091D20220FB90F99093D20277
:103CC0000C94201F0E94491E8091D2020C94521D18
:103CD000FC01DB0112968C918823F9F0EC5BFC452A
:103CE000E730F105D8F4EE59FF4F0C94DC2B83E05C
:103CF00001C080E00E94621E80E008950E94D21DF3
:103D0000FBCF0E94AF1DF8CF0E94191EF5CF0E9475
:103D1000201EF2CF0E947D1DEFCF81E00895269AEC
:103D20002E9808952E9808958F929F92AF92BF92E9
:103D3000CF92DF92EF92FF920F931F93CF93DF9377
:103D40008C0180918600909187006CE070E00E9469
:103D5000922B6017710730F0C80169E070E00E9493
:103D6000922B60C08091860090918700E090860041
:103D7000F0908700E0918600F0918700C6E0D0E0E7
:103D8000BE010E94922B20E030E0060F171F211D7C
:103D9000311D4801590185E0880C991CAA1CBB1CE7
:103DA0008A95D1F7C701BE010E94922B6F01E12CC9
:103DB000F12CA7019601260F371F411D511DC5018A
:103DC000B4010E94BA2B69017A01E0918600F0915A
:103DD0008700CA01B9010E94822B9B01AC01DF015F
:103DE0000E94002C9B01AC01C701B6010E94822BEE
:103DF000DC01CB012FE0B695A795979587952A957D
:103E0000D1F7009186001091870020E030E008177C
:103E100019072A073B0728F46091860070918700F4
:103E2000CB01BC01CB01DF91CF911F910F91FF908E
:103E3000EF90DF90CF90BF90AF909F908F900895BC
:103E4000CF93C82F843050F4811109C08091800035
:103E50008F7D809380000E94921E06C0C3E08091F7
:103E60008000806280938000A0918600B0918700DE
:103E70002C2F30E00E94EA2B23E030E040E050E0BD
:103E80000E94BA2BB42FA32F922F8827892F9A2F05
:103E9000AB2FBB270E94941E90938B0080938A00C7
:103EA000CF9108950895109282021092810210928B
:103EB0008302EFE6F0E08081816080830895EFE681
:103EC000F0E080818E7F80830E945F1D0C94201F14
:103ED0001F920F920FB60F9211240F931F932F93DF
:103EE0003F934F935F936F937F938F939F93AF9382
:103EF000BF93CF93EF93FF938091200191E0980FB0
:103F0000823019F09093200155C081E08093200108
:103F10000E94891DC82F00918102109182020F5FBB
:103F20001F4F0E94891D28E7829FB0011124C801FC
:103F30000E94922B909382028093810228E7C29F75
:103F4000B0011124660F672F661F770B71950E94D1
:103F5000922B6F7780918302823019F4603451F490
:103F600004C0813039F46F3729F480916F008E7F5F
:103F700080936F00E62FF0E0E356FD4FC49100916F
:103F80008600109187000E945F1D282FC09FC001EE
:103F9000C19F900D11246DEF72E00E94922B269F1D
:103FA000C001279F900D11240E94941E90938B00B6
:103FB00080938A00FF91EF91CF91BF91AF919F9134
:103FC0008F917F916F915F914F913F912F911F91B1
:103FD0000F910F900FBE0F901F9018950E948F1E8B
:103FE00082E28093800089E1809381008FEF9FEFD0
:103FF00090938700809386000E948C1D0E94841DF0
:1040000081110C94531F0895239A25B1277F35B150
:1040100038604FB7F894FC01CB01880F991F680FE7
:10402000791F6E0F7F1FE617F70789F0819198E0DF
:1040300035B9000000C087FF25B9880F000000C017
:1040400000C000C025B900C09A9591F7ECCF4FBFD2
:104050008FE594E00197F1F700C000000895CF9339
:10406000DF93EC01FB018281882309F43CC1C43059
:10407000FDE5DF0760F4CB3F9CE5D90788F49E019E
:1040800022503C452431310508F02EC109C0C2360A
:10409000EDE5DE0729F0C63AFDE5DF0709F024C1AA
:1040A0000E946B0E9093B6028093B502C1318CE5ED
:1040B000D80709F4C6C008F042C0C930ECE5DE07F5
:1040C00009F49BC000F5C5308CE5D80709F485C01C
:1040D00078F4C330ECE5DE0709F478C008F07AC064
:1040E000C230DC4509F0F5C08091B5028160EFC0B7
:1040F000C7309CE5D90709F478C008F07AC08091F0
:10410000B5028061E4C0CD30FCE5DF0709F487C06B
:1041100058F4CB309CE5D90709F479C008F07BC08E
:104120008091B50288606FC0CF30FCE5DF0709F4ED
:1041300080C008F082C08091B502877FC8C0CE3FA2
:104140009CE5D90709F471C000F5C531FCE5DF072E
:1041500009F485C068F4C3319CE5D90709F475C03A
:1041600008F095C00E941E088091B5028F77AFC0FD
:10417000CC3FFCE5DF07A9F108F054C0CB3FDC459C
:1041800009F0A7C08091B60240C0C230EDE5DE075D
:1041900009F489C058F4C1158DE5D80709F45AC04F
:1041A00008F069C08091B60282602FC0C236EDE58A
:1041B000DE0709F47CC0C63AFDE5DF0709F481C0DB
:1041C000C330DD4509F085C080E06EC08091B50246
:1041D00082607DC08091B50216C08091B502886072
:1041E00076C08091B60282604FC08091B502806235
:1041F0006EC08091B50280646AC00E941E088091E2
:10420000B502806864C0846062C081603DC08091F6
:10421000B5028E7F5CC08091B5028D7F58C08091C1
:10422000B50216C08091B60218C08091B6028D7F8B
:104230002BC08091B5028F7E4AC08091B5028F7DE0
:1042400046C08091B5028F7B42C08091B502877FC6
:104250008B7F3DC08091B6028D7F8E7F15C080918F
:10426000B50282FB222720F991E0922790FB82F988
:1042700090FB83F92CC08091B602982F9095917095
:104280008E7F892B90FB81F98093B60222C00E9419
:104290001E088091B50287FB222720F991E0922722
:1042A00090FB87F914C081E00E94020F12C0809138
:1042B000B50284FB222720F991E0922790FB84F934
:1042C00006C08091B502982F909590FB80F980935D
:1042D000B5028091B5029091B6020E947C0E0E94B8
:1042E0001E0880E001C081E0DF91CF910895CF9357
:1042F000DF9386319C4541F5EB010E946F0D982FAD
:104300008A812091020130910301882379F09A7A01
:1043100081E009F480E080938402911102C069E297
:1043200001C065E3C9010E946D230AC08091840227
:10433000811102C069E201C065E3C9010E947823CE
:104340000E94B10D80E001C081E0DF91CF9108951E
:104350000F931F93CF93DF93C42FD22FFC01828141
:104360008823C9F0409387020E94302490938602EC
:104370008093850280E28C0F883008F057C0C770A8
:1043800081E001C0880FCA95EAF7DF91CF911F91B4
:104390000F910C947B0580918702481330C0809167
:1043A0008502909186020E944824883C910538F548
:1043B00010E21D0FCD17B9F080E28C0F883040F469
:1043C000C77081E001C0880FCA95EAF70E94820594
:1043D000183028F581E09D2F977001C0880F9A95BD
:1043E000EAF70E947B05802F0E9472051830F0F4D6
:1043F000D77081E001C0880FDA95EAF70AC080E241
:104400008C0F883098F4C77081E001C0880FCA957E
:10441000EAF7DF91CF911F910F910C948205802FC5
:10442000DF91CF911F910F910C947205DF91CF9185
:104430001F910F9108950F939C01CB01243F4CE5F0
:10444000340731F188F4293DFCE53F07D9F02A3DD6
:104450004CE5340779F1283D3C45A9F506E221EE0B
:1044600041EE68ED7CE52BC0263FFCE53F07E1F01F
:10447000A8F0273F3C4539F507E225EE46EE67EF09
:104480007CE51DC007E225EE45EE69ED7CE517C031
:1044900006E221EE40EE64EF7CE511C007E225EE76
:1044A00044EE65EF7CE50BC006E221EE42EE66EFDE
:1044B0007CE505C008E221E045EE6AED7CE50E945E
:1044C000A82180E008C0FC018281882319F01092A5
:1044D000870201C081E00F9108959093BF018093FE
:1044E000BE01089590938D0280938C020895E0910F
:1044F0008C02F0918D02309721F00190F081E02D37
:10450000099480E00895E0918C02F0918D0230973B
:1045100099F020912D01222359F02091B50227FF17
:1045200007C0DC012C9111962C93119726E02C9357
:104530000280F381E02D09940895E0918C02F091BE
:104540008D02309739F022E0DC012C930480F58154
:10455000E02D0994089520918A0230918B0228174A
:10456000390771F090938B0280938A02E0918C025C
:10457000F0918D02309721F00680F781E02D0994AB
:10458000089520918802309189022817390771F027
:104590009093890280938802E0918C02F0918D02C1
:1045A000309721F00084F185E02D09940895FC01F5
:1045B000329680912D01882331F08091B50287FFDA
:1045C00002C09EE101C096E080E0915028F0219168
:1045D0002223D9F38F5FF9CF0895662351F12091FB
:1045E0002D012223E9F02091B50227FF19C0462FA3
:1045F0004695469546954E31E0F4677021E030E0EF
:1046000002C0220F331F6A95E2F7FC01E40FF11D8F
:10461000828190E02823392381E0232B69F409C0AB
:10462000FC01329608962191621729F0E817F907E4
:10463000D1F780E0089581E008959C01FC01329655
:104640009FEF80E04191461789F09F3F19F4411197
:1046500001C0982F8F5F8630A9F79F3F39F0F9018D
:10466000E90FF11D97FDFA956283089508959C0165
:104670002A5F3F4FFC014281461301C0128201961E
:1046800082179307B9F70895262F26952695269524
:104690002E3168F4FC01E20FF11D677021E030E07B
:1046A00001C0220F6A95EAF78281282B22830895A0
:1046B000262F2695269526952E3170F4FC01E20FC3
:1046C000F11D677021E030E001C0220F6A95EAF722
:1046D0002095828128232283089520912D01222371
:1046E00029F02091B50227FD0C9444230C941D233E
:1046F00020912D01222329F02091B50227FD0C9451
:1047000058230C94372320912D01FC01329622234B
:1047100031F08091B50287FF02C08EE101C086E0D2
:10472000DF011D928A95E9F7089508950C94952369
:1047300083E080938E020C949623811102C081E065
:1047400001C082E080938E020C9496230C949D23EA
:1047500081E080938E020C9496230C94A8230895F4
:104760000C94AF230C94B0230C94AF230C94AF2380
:104770000C94AF23CF930E94B6230E94FA120E949A
:10478000B423C0E08C2F0E942D12811104C0CF5F92
:10479000C530C1F701C081E0CF91089508951F92FF
:1047A0000F920FB60F9211248F939F93AF93BF93E5
:1047B00080918F02811113C08091D3029091D40215
:1047C000A091D502B091D6024196A11DB11D809352
:1047D000D3029093D402A093D502B093D602BF9196
:1047E000AF919F918F910F900FBE0F901F901895D2
:1047F0008091DB02843031F10E94C50310928F0258
:1048000020E488E190E00FB6F894A89580936000CA
:104810000FBE2093600083B7817F846083BF83B71E
:10482000816083BF7894889583B78E7F83BF0FB6EE
:10483000F894A89580916000886180936000109240
:1048400060000FBE08950E941E080C94CE0382E003
:1048500084BD93E095BD9AEF97BD80936E00089557
:104860002FB7F8948091D3029091D402A091D502F1
:10487000B091D6022FBF08952FB7F8946091D3025C
:104880007091D4028091D5029091D6022FBF0895E5
:104890009C014FB7F8948091D3029091D402A091DB
:1048A000D502B091D6024FBF821B930B0895789426
:1048B0001F920F920FB60F9211248F939F93AF9375
:1048C000BF938091D3029091D402A091D502B09170
:1048D000D6020196A11DB11D8093D3029093D402FC
:1048E000A093D502B093D602BF91AF919F918F91C3
:1048F0000F900FBE0F901F90189581E08093E000FD
:1049000080E28093D8001092C9008FE19EE4019765
:10491000F1F700C0000087E090EBDC018093E40237
:104920009093E502A093E602B093E7029CE088E151
:104930000FB6F894A895809360000FBE9093600026
:10494000FFCF8091B3020895089522E02093E900FB
:104950002FEF3091E800215035FD06C035ED3A9536
:10496000F1F700002111F5CF2091E80025FF0BC0E1
:1049700040E050E066E070E00E94E4268091E800AC
:104980008E778093E8000895CF93DF9320912D01D7
:10499000222339F02091B50227FF03C060E222E014
:1049A00002C068E021E02093E9002FEF3091E80099
:1049B000215035FD06C035ED3A95F1F70000211183
:1049C000F5CF2091E80025FF1DC0EC0180912D015D
:1049D000811105C040E050E068E070E003C070E085
:1049E00040E050E0CE010E94E4268091E8008E77FE
:1049F0008093E80080E2FE01A3E9B2E001900D920D
:104A00008A95E1F7DF91CF9108958093900270939A
:104A10009202609391028091DB02843001F582E082
:104A20008093E9008FEF9091E800815095FD06C0DA
:104A300095ED9A95F1F700008111F5CF8091E8008E
:104A400085FF0DC040E050E063E070E080E992E057
:104A50000E94E4268091E8008E778093E800089514
:104A6000BC0184E00C940525BC0183E00C94052571
:104A70008091DA02811109C00E9475280E94D22813
:104A80008091E20084608093E20008951092DA023F
:104A900008950C94AD236091D70281E0611101C0AB
:104AA00080E00C9498239091DB0281E0943009F02F
:104AB00080E06091D7020C949D2342E061EC81E09C
:104AC0000E94EE2742E261EC82E00E94EE27909184
:104AD000DB0281E0943009F080E06091D7020C9411
:104AE000A6238091DD02833009F461C030F4813067
:104AF00071F0823009F49AC008958A3009F486C0B2
:104B00008B3009F46CC0893009F0A8C020C08091B6
:104B1000DC02813A09F0A2C08091E800877F80938F
:104B2000E8008091E0029091E102892B21F460E29B
:104B300083E992E003C060E080E090E070E00E94D2
:104B40002F278091E8008B778093E800089580916B
:104B5000DC02813209F082C08091E0029091E10292
:104B6000029708F07BC08091E800877F8093E8007F
:104B70008091E80082FD05C08091DB028111F8CFB1
:104B80006DC02091F3008091F20090E0922B02978B
:104B900031F48091F100813011F0863021F4809160
:104BA000F1008093B3028091E8008B7753C080912D
:104BB000DC02813A09F052C08091E0029091E1025A
:104BC000892B09F04BC08091E800877F8093E80033
:104BD0008091E80080FFFCCF80912D0136C080914C
:104BE000DC028132D9F58091E0029091E102892BBB
:104BF000A9F58091E800877F8093E8000E94232830
:104C00008091DE0280932D010C941E088091DC02BD
:104C1000813221F58091E800877F8093E8000E942F
:104C200023288091DF028093B40208958091DC02F2
:104C3000813AA1F48091E800877F8093E800809119
:104C4000E80080FFFCCF8091B4028093F100809156
:104C5000E8008E778093E8000C942328089584B7A9
:104C6000877F84BF0FB6F894A89580916000886113
:104C700080936000109260000FBE90E080E80FB655
:104C8000F89480936100909361000FBE0C94A82368
:104C90000E9475280E94D228E2EEF0E080818460B4
:104CA000808378940C94672B81E291E00C947222BB
:104CB0008091DB028530A9F48091DB02853079F4A4
:104CC0000E94F8238091D9028823B1F30E94BA236D
:104CD000882391F30E94CE260E941E08EDCF0C94EB
:104CE0002324089508950C947526292F3327233003
:104CF0003105C9F060F42130310581F022303105F1
:104D000009F044C08BE390E027E434E043C0213253
:104D10003105E1F02232310549F138C082E190E0FD
:104D200022E834E037C099278130910549F028F016
:104D3000029761F5EDE1F4E005C0E3E4F4E002C0C0
:104D4000E7E2F4E0849190E09F0124C061157105D1
:104D500041F061307105D1F489E090E022E734E060
:104D600019C089E090E029E534E014C061157105AF
:104D700041F06130710551F486EB90E024E934E0B4
:104D800009C080E490E02AE435E004C080E090E0CF
:104D900020E030E0FA0131832083089580E189BD6D
:104DA00082E189BD09B400FEFDCF8091D8008F7DDE
:104DB0008093D8008091E00082608093E000809131
:104DC000E00081FDFCCF0895CF92DF92EF92FF9239
:104DD0000F931F93CF93DF93EC018B017A010E9415
:104DE0004228811133C0E114F10439F0F7018081C8
:104DF0009181081B190BC80FD91FC12CD12C01158B
:104E0000110519F18091E80085FD16C08091E80038
:104E10008E778093E800E114F10449F0F701808176
:104E20009181C80ED91ED182C08285E00FC00E9438
:104E30004228882321F30AC089918093F100015010
:104E40001109FFEFCF1ADF0ADACF80E0DF91CF91AF
:104E50001F910F91FF90EF90DF90CF9008952091D8
:104E6000E2023091E3022617370748F06115710519
:104E700039F42091E8002E772093E80001C0B901B1
:104E8000FC0120E06115710579F18091DB02882336
:104E9000F1F18530F1F18091E80083FD3CC0809113
:104EA000E80082FD2EC08091E80080FFEBCF2091CA
:104EB000F3008091F20090E0922B6115710551F0A2
:104EC0008830910538F421912093F10061507109E7
:104ED0000196F3CF21E0089709F020E08091E800E7
:104EE0008E778093E800CECF2111CFCF0AC080917A
:104EF000DB02882361F0853061F08091E80083FD5A
:104F00000AC08091E80082FFF2CF80E0089582E03D
:104F1000089583E0089581E008952091E2023091A0
:104F2000E3022617370748F06115710539F420911F
:104F3000E8002E772093E80001C0B901FC0120E0D1
:104F40006115710591F18091DB02882309F440C05D
:104F5000853009F43FC08091E80083FD3DC0809119
:104F6000E80082FD2FC08091E80080FFE9CF20910A
:104F7000F3008091F20090E0922B6115710559F0D9
:104F80008830910540F424912093F10031966150CE
:104F900071090196F2CF21E0089709F020E0809195
:104FA000E8008E778093E800CBCF2111CCCF0AC0E8
:104FB0008091DB02882361F0853061F08091E80008
:104FC00083FD0AC08091E80082FFF2CF80E008955F
:104FD00082E0089583E0089581E00895982F973046
:104FE00068F59093E900981739F07091EC002091E2
:104FF000ED005091F00003C0242F762F50E021FDEA
:1050000002C09F5FECCF3091EB003E7F3093EB000E
:105010003091ED003D7F3093ED003091EB00316039
:105020003093EB007093EC002093ED005093F00070
:105030002091EE0027FDE5CF80E008958F708093EA
:10504000E90081E008958091DC0287FF11C0809122
:10505000E80082FD05C08091DB028111F8CF11C00C
:105060008091E8008B770BC08091DB02882349F0A8
:105070008091E80080FFF8CF8091E8008E778093E0
:10508000E80008952091E4003091E50095E6409114
:10509000EC00842F817040FF23C08091E80080FDE8
:1050A0001DC08091DB02882399F0853099F08091B2
:1050B000EB0085FD11C04091E4005091E5002417FC
:1050C000350729F3915011F09A01E1CF84E008955A
:1050D00082E0089583E0089581E0089580E00895D6
:1050E0004091E80042FFDDCF08950E94E3280E942E
:1050F000EB28E0EEF0E0808181608083E8EDF0E075
:1051000080818F77808319BCA7EDB0E08C918E7F72
:105110008C9380818F7E80831092DA0208950F93A2
:105120001F93CF93DF930E94E3280E94EB28C8EDE2
:10513000D0E088818F7788838881806888838881A0
:105140008F7D888319BC1092DB021092D7021092D7
:10515000D9021092D80200EE10E0F80180818B7F16
:10516000808388818160888342E060E080E00E94E3
:10517000EE27E1EEF0E080818E7F8083E2EEF0E0CA
:10518000808181608083808188608083F801808154
:105190008E7F8083888180618883DF91CF911F918A
:1051A0000F910895E8EDF0E080818F7E8083E7ED38
:1051B000F0E080818160808384E082BF81E0809321
:1051C000DA020C948F28E8EDF0E080818E7F8083F6
:1051D0001092E20008951092DA001092E100089512
:1051E0001F920F920FB60F9211242F933F934F935C
:1051F0005F936F937F938F939F93AF93BF93EF933F
:10520000FF938091E10082FF0BC08091E20082FF5A
:1052100007C08091E1008B7F8093E1000E94662BA4
:105220008091DA0080FF1FC08091D80080FF1BC0F2
:105230008091DA008E7F8093DA008091D90080FF20
:105240000DC080E189BD82E189BD09B400FEFDCFBA
:1052500081E08093DB020E94382505C019BC1092C2
:10526000DB020E9446258091E10080FF19C08091F9
:10527000E20080FF15C08091E2008E7F8093E20003
:105280008091E20080618093E2008091D80080628A
:105290008093D80019BC85E08093DB020E944B25E7
:1052A0008091E10084FF30C08091E20084FF2CC037
:1052B00080E189BD82E189BD09B400FEFDCF809106
:1052C000D8008F7D8093D8008091E1008F7E8093FD
:1052D000E1008091E2008F7E8093E2008091E20005
:1052E00081608093E2008091D702882311F084E0EE
:1052F00007C08091E30087FD02C081E001C083E028
:105300008093DB020E9453258091E10083FF29C036
:105310008091E20083FF25C08091E100877F809328
:10532000E10082E08093DB021092D7028091E100DD
:105330008E7F8093E1008091E2008E7F8093E20077
:105340008091E20080618093E20042E060E080E0D2
:105350000E94EE278091F00088608093F0000E9408
:105360004925FF91EF91BF91AF919F918F917F91CF
:105370006F915F914F913F912F910F900FBE0F90C2
:105380001F9018951F920F920FB60F9211242F9312
:105390003F934F935F936F937F938F939F93AF93BD
:1053A000BF93CF93DF93EF93FF93C091E900CF704A
:1053B0008091EC00D82FD17080FDD0E81092E900E8
:1053C0008091F000877F8093F00078940E94062AF5
:1053D0001092E9008091F00088608093F000CD2B5E
:1053E000CF70C093E900FF91EF91DF91CF91BF9112
:1053F000AF919F918F917F916F915F914F913F916D
:105400002F910F900FBE0F901F9018951F93CF9361
:10541000DF93CDB7DEB7AA970FB6F894DEBF0FBE05
:10542000CDBFECEDF2E08091F100819322E0E43E0B
:10543000F207C9F70E9471258091E80083FF2EC111
:105440008091DC029091DD02492F50E04A305105F5
:1054500008F024C1FA01E759FF4F0C94DC2B803887
:1054600021F0823809F01AC108C08091D8029091C9
:10547000D902992389F082600FC08091E0028F7079
:10548000873008F00BC18093E9008091EB0085FB29
:10549000882780F91092E9009091E800977F909317
:1054A000E8008093F1001092F100D1C0282F2D7FE9
:1054B00009F0F4C0882319F0823061F0EFC08091C8
:1054C000DE02813009F0EAC0933009F080E0809379
:1054D000D9022EC08091DE0281112AC08091E002A3
:1054E0008F702FEF280F263008F0D8C08093E90086
:1054F0002091EB0020FF1CC0933021F48091EB0041
:10550000806214C09091EB0090619093EB0021E0D9
:1055100030E0A90102C0440F551F8A95E2F740937D
:10552000EA001092EA008091EB0088608093EB0023
:105530001092E9008091E800877F8093E8000E9444
:105540002328ACC08111AAC01091DE021F77809180
:10555000E3008078812B8093E3008091E800877FCF
:105560008093E8000E9423288091E80080FFFCCF10
:105570008091E30080688093E300111102C082E013
:1055800001C083E08093DB0289C08058823008F03C
:1055900085C08091DE029091DF028C3D53E095073B
:1055A00079F583E08A838AE289834FB7F894DE0134
:1055B000139620E03EE051E2E32FF0E050935700D5
:1055C000E49120FF03C0E295EF703F5FEF708E2FF4
:1055D00090E0EA3010F0C79601C0C0968D939D937D
:1055E0002F5F243149F74FBF8091E800877F809378
:1055F000E8006AE270E0CE0101960E942F2716C0F3
:105600006091E0027091E102AE014F5F5F4F0E9436
:105610007326BC01892B09F441C09091E800977F63
:105620009093E80089819A810E948D278091E800FB
:105630008B778093E80032C0803881F58091E80054
:10564000877F8093E8008091D7028093F10080915A
:10565000E8008E7772CF811121C08091DE02909197
:10566000DF0299270297D4F48091E800877F809326
:10567000E8008091DE028093D7020E942328809167
:10568000D702811106C08091E30087FD02C081E04E
:1056900001C084E08093DB020E945D258091E800D8
:1056A00083FF0AC08091E800877F8093E8008091A3
:1056B000EB0080628093EB00AA960FB6F894DEBFF1
:1056C0000FBECDBFDF91CF911F9108950895CF9365
:1056D0008091DB028823A1F0C091E900CF70909106
:1056E000EC00892F817090FD80E8C82B1092E900B2
:1056F0008091E80083FD0E94062ACF70C093E900E4
:10570000CF910895DB018F939F930E94002CBF914E
:10571000AF91A29F800D911DA39F900DB29F900D00
:1057200011240895AA1BBB1B51E107C0AA1FBB1F70
:10573000A617B70710F0A61BB70B881F991F5A951D
:10574000A9F780959095BC01CD01089597FB072E90
:1057500016F4009407D077FD09D00E94922B07FC25
:1057600005D03EF4909581959F4F08957095619571
:105770007F4F0895A1E21A2EAA1BBB1BFD010DC08D
:10578000AA1FBB1FEE1FFF1FA217B307E407F507F1
:1057900020F0A21BB30BE40BF50B661F771F881FCD
:1057A000991F1A9469F760957095809590959B0163
:1057B000AC01BD01CF010895EE0FFF1F0590F491DC
:1057C000E02D09940E94EA2B332312F48A1B9B0BD1
:1057D0000C94FB2BA29FB001B39FC001A39F700D3F
:1057E000811D1124911DB29F700D811D1124911DE9
:1057F00008950E94EA2BB7FF0895821B930B08952A
:105800000E94EA2BA59F900DB49F900DA49F800D40
:10581000911D11240895B7FF0C94002C0E94002CB8
:10582000821B930B0895FC014150504030F00190D1
:105830000616D1F73197CF01089588279927089543
:10584000FB01DC0104C08D910190801921F44150CD
:105850005040C8F7881B990B0895F999FECF92BD67
:1058600081BDF89A992780B50895A6E1B0E044E09B
:1058700050E00C94672CA8E1B0E042E050E00C94BA
:10588000672C262FF999FECF92BD81BDF89A01971A
:1058900000B4021639F01FBA20BD0FB6F894FA9A78
:1058A000F99A0FBE08950396272F0E94422C0E945A
:1058B000412C252F0E94422C242F0C94422C01961F
:1058C000272F0E94422C0C94412CDC01CB01FC01BF
:1058D000F999FECF06C0F2BDE1BDF89A319600B449
:0E58E0000D9241505040B8F70895F894FFCF54
:1058EE00C8003302280850011E0A140101010200EB
:1058FE000400040401191A1B1C1D1E1F2021220660
:10590E0001A124C424A52434253025A42401E200B9
:10591E00E900EA00B500B600B700CD008301CC0067
:10592E008A019201940121022302240225022602F9
:10593E0027022A02B300B4006F007000818283E256
:10594E0000E900EA00B500B600B700CD008301CC37
:10595E00008A0192019401210223022402250226CB
:10596E000227022A02B300B4006F00700081828306
:10597E006667949637C69091950001020202020660
:10598E0006060909090909090F0F0F0F0F0F151543
:0E599E0015181919191919191919191923248D
:00000001FF
